:100000000C945A010C9477010C9492010C94770192
:100010000C9477010C9477010C94C4180C9477011C
:100020000C9477010C9477010C9477010C94770170
:100030000C9477010C9477010C944C190C94770173
:100040000C9477010C9477010C9477010C94770150
:100050000C9477010C9477010C9477010C94770140
:100060000C9477010C94770181058105AD05AD05F0
:10007000150633064B074B073E06D706E806E8068B
:10008000290014001A000800150017001C001800B1
:100090000C0012001300394204001600070009008A
:1000A0000A000B000D000E000F002800E1001D00EB
:1000B0001B00060019000500110010003600370073
:1000C000E500E000E300E2002C0000002C0000004E
:1000D000650001512A00E400005C1E001F002000A2
:1000E00021002200230024002500260027000251C1
:1000F0003A003B003C003D003E003F002D002E003A
:1001000033003400E100400041004200430044005D
:1001100045003600370038003800E000E300E20018
:100120002C0000002C000000650001004C00E400E1
:10013000005C1E005200C35CC45C2200230024004B
:100140002500260027000100500051004F00C65C2A
:10015000C75CC85CC95CCA5CCB5C280001000100BC
:100160000100010001000100010001000100520036
:1001700001000100010001002C0000002C00000023
:10018000500051004C004F0009023B00020100A04A
:1001900032090400000103010100092101010001ED
:1001A0002240000705810308000109040100010342
:1001B000000000092101010001227B0007058303E3
:1001C0000800011201100100000008EDFE0000020D
:1001D00000010200010E0348006E00610068003457
:1001E00000300000000E0348006E00610068004B04
:1001F00000420000000403090405010902A1018571
:10020000020901A100050919012908150025019518
:1002100008750181020501093009311581257F9595
:10022000027508810609381581257F9501750881B9
:1002300006050C0A38021581257F9501750881068F
:10024000C0C005010980A101850319012AB7001565
:100250000126B700950175108100C0050C0901A1A8
:1002600001850419012AA002150126A00295017535
:10027000108100C005010906A101050719E029E761
:100280001500250195087501810295017508810306
:100290000507190029FF150026FF0095067508813E
:1002A000000508190129059505750191029501754B
:1002B000039103C011241FBECFEFD8E0DEBFCDBF36
:1002C00011E0A0E0B1E0ECE1FAE302C005900D928C
:1002D000AC38B107D9F723E0ACE8B1E001C01D921A
:1002E000AC32B207E1F70E9427130C940C1D0C945A
:1002F0000000A82FB92F80E090E041E050EA60951F
:1003000030E009C02D9182279795879510F08427BA
:100310009527305EC8F36F5FA8F30895EADF8D93E9
:100320009D930895CF93CFB7CF93DF93C3954B9B06
:10033000E9F74B9B10C04B9B0EC04B9B0CC04B9BDB
:100340000AC04B9B08C04B9B06C0C0910303C395DA
:10035000C09303038EC06F93C0910203DD27C65F75
:10036000DC4F2F9365E54B9B03C02F916F91E1CF3D
:100370000F931F934F9320E040E15F9309B10C70FE
:1003800003FB27F93F9350E03BE039C01C70406409
:100390002F77012F5F5F1EC0406819B11C702F7747
:1003A00052501FC0406409B12F770C70D1F15F5FCC
:1003B00000C023C0406219B12F771C7091F15F5FBC
:1003C00000C025C00C701027515012F45D5F000072
:1003D000115027952C3F19B1C8F61C700127015008
:1003E00027952C3FC8F64227499309B10C70102776
:1003F0004F73115027952C3FA8F64695469519B195
:100400001C7079F00127015027952C3F98F66B5A04
:1004100060F3315009B1B0F600C012E01CBB0027F8
:100420001CC03B503195C31BD04012E01CBB08815F
:10043000033C21F10B3411F12091FF021981110FBE
:100440001213EDCF4A81441F093679F10D3211F0B4
:10045000013E29F74F7009F0042F009308033F91E4
:100460005F914F911F910F912F916F91CCB3C1FD6F
:100470005DCFDF91CF91CFBFCF9118952091080329
:10048000222369F310910603112309F049C0343087
:100490000AF448C03093060320930103109102032D
:1004A0003BE0311B309302033DC000910603013055
:1004B000BCF50AE54F7049F43091190134FD33C0A1
:1004C00000931901CCEDD2E032C0433059F04430F2
:1004D00091F03091E70234FD26C00093E702C8EEA8
:1004E000D2E025C03091200334FD1DC000932003CD
:1004F000C1E2D3E01CC03091F30234FD14C000937C
:10050000F302C4EFD2E013C0052710E000C00000E2
:100510000BB91AC0052710E0221F1DC010E021C032
:100520004AE502C032ED432FC4E1D0E032E01AB117
:100530001C605B9A0BB11AB95CE020E865E320FF10
:1005400005270BB9279517951C3FF0F66695B8F768
:10055000B1F720FF05270BB9279517951C3FD0F65B
:100560002795179517FF052700001C3F0BB9B0F61C
:1005700029913A9519F7037F10910703110FC6517E
:10058000D0400BB911F01093FF0212E01CBB0860C1
:100590001AB1137F402F437F54E05A95F1F70BB9FE
:1005A0001AB94BB95CCF81E0089581E008950C94AD
:1005B000D50208950C94D9021F93CF93DF9300D0F6
:1005C00000D01F92CDB7DEB749835A836B83309139
:1005D0008F0189819A81311114C0662359F0222339
:1005E00049F00E948809182F682F89819A810E94FA
:1005F000310903C00E945C09182F69817A81812F1B
:1006000004C00E94880969817A810F900F900F9031
:100610000F900F90DF91CF911F910C94AF10FC01C0
:10062000262F408151816281738184810C94DC0288
:1006300081E00895CF93DF93EC0160E00E940F0307
:10064000BE01DF91CF910C94DA020C94DE110C9470
:10065000DA1108950E94DB070E9429032FEF84E33B
:100660009CE0215080409040E1F700C000000C94D5
:1006700072190F931F93CF93DF938C0161E00E9457
:100680000F03EC01B8010E94D7028823F1F1B801F1
:10069000CE010E94A9178823C1F1B801CE010E94A2
:1006A000BD15882391F1B801CE010E94051788235A
:1006B00061F1F8018281882309F1CB358DE5D807F6
:1006C000C1F050F4C115FCE5DF0781F0CF3DDC45FA
:1006D000A9F40E94B90E19C0CC35EDE5DE0761F032
:1006E000CD35DD4559F40E94020E08C00E942A0350
:1006F0000CC00E940B0E02C00E940E0EC801DF91BA
:10070000CF911F910F910C94D30280E0DF91CF9194
:100710001F910F9108950E94A6180C94A4030E94A3
:10072000A7030C94AC1808950C94930381E00895EA
:100730000C9496030895CF93C82F0E9494038C2F96
:100740000E949803CF91089580E00C949B030E942F
:1007500005180C949B030E94051890918E0189172F
:1007600021F080938E010C949B030895CF93DF9327
:10077000CDB7DEB72B970FB6F894DEBF0FBECDBF57
:100780004F83588769877A878B8761110E944E0D46
:100790009E012F5F3F4F86E0F90111928A95E9F79C
:1007A00085E0FE013796D90101900D928A95E1F717
:1007B00089819A814C815D81452B31F09F3F31F4D5
:1007C00091E08F3F19F403C091E001C090E090FFE9
:1007D00009C049815A816B817C818D819E810E94F3
:1007E0006F0C05C0C9010E9418038111F2CF2B962E
:1007F0000FB6F894DEBF0FBECDBFDF91CF91089545
:10080000FC01808191810E94CA090895CF938823B9
:1008100009F4A4C0C82F8238C1F40E94051881FDD4
:100820009DC069E380910201909103010E94981894
:100830000E94700D2FEF81EE94E021508040904097
:10084000E1F700C0000069E319C0833801F50E9498
:10085000051880FD83C063E580910201909103013A
:100860000E9498180E94700D2FEF81EE94E02150A5
:1008700080409040E1F700C0000063E580910201F4
:10088000909103010E949A18CF910C94700D8438B6
:10089000C1F40E94051882FD61C067E480910201E5
:1008A000909103010E9498180E94700D2FEF81EE25
:1008B00094E0215080409040E1F700C0000067E4E0
:1008C000DDCF8CEF8C0F813AD0F46C2F8091020138
:1008D000909103010E946218882349F06C2F809147
:1008E0000201909103010E949A180E94700D6C2FD2
:1008F00080910201909103010E949818C5CF80E277
:100900008C0F883048F4C77081E001C0880FCA9509
:10091000EAF70E94310DB8CFEBE5EC0FE33040F47D
:10092000F0E0E85BFE4F808190E0CF910C942A18B4
:10093000E8E5EC0FE73150F4F0E0EE0FFF1FE65E64
:10094000FE4F80819181CF910C944018CD3E30F0C4
:100950008C2F0E94AC13CF910C947E14CF910895EC
:10096000882309F464C0823879F40E94051881FF55
:100970005EC069E380910201909103010E94981882
:100980000E94700D69E310C08338B1F40E9405180D
:1009900080FF4DC063E580910201909103010E94A8
:1009A00098180E94700D63E58091020190910301F7
:1009B0000E949A180C94700D843879F40E940518DE
:1009C00082FF35C067E480910201909103010E948B
:1009D00098180E94700D67E4E7CF9CEF980F913A4A
:1009E00010F4682FE1CF90E2980F983050F48770A0
:1009F00091E001C0990F8A95EAF7892F0E94370D7F
:100A0000D9CF9BE5980F933020F480E090E00C94D0
:100A10002A1898E5980F973120F480E090E00C9424
:100A200040188D3E20F00E9407140C947E14089507
:100A30001F93CF93DF93182FEB010E94060420979A
:100A400041F08FE99FE00197F1F700C00000219786
:100A5000F6CF812FDF91CF911F910C94B004893391
:100A600019F060E070E002C060E570E00C941805D9
:100A7000882321F00E94310D0C94700D0895882375
:100A800021F00E94370D0C94700D0895CF92DF92E3
:100A9000EF92FF920F931F93CF93DF937C01D62F9A
:100AA000C72FFC011281058102950F700E94270D4E
:100AB0008823B9F01123A9F08C2F807F803421F096
:100AC00080E28D0F883068F08091C70282FD09C0F6
:100AD00082E00E94D00D0E94270D91E0D82ED926E9
:100AE00001C0D12CCC2EC2948FE0C8228C2D90E076
:100AF0008C30910508F0CFC1FC01EC5CFF4F0C94E9
:100B0000A31C8C2F807FCF70882311F0C295C07FEB
:100B1000112399F0CC2309F4AAC180E28D0F88300B
:100B200010F0D11104C08C2F0E94310D03C08C2F06
:100B30000E94410D0E94700D9AC18D2F0E94B00439
:100B4000CC2309F4A8C180E28D0F883038F1DD2371
:100B500029F18C2F0E94470D24C08C2F807FCF70ED
:100B6000803211F0C295C07FDD2319F0D130A1F1A0
:100B70003DC08091C70282FF17C0112349F0CC23EA
:100B800029F08C2F0E94310D0E94700D80E070C101
:100B900080E00E94B004CC2309F47DC18C2F0E9418
:100BA000370D0E94700D77C1112371F0002341F0C1
:100BB000013031F40E94510D8C2B0E94590D6BC1F4
:100BC0000E94510D8C2B1DC0002319F0013009F437
:100BD00062C10E94660D25C0112321F0063008F085
:100BE0005AC10EC0053008F056C11BC0112361F078
:100BF000002331F0F701858180FF39C18F70858333
:100C00008C2F0E94380547C1002359F0D93309F0D1
:100C10003FC1FFEF07EE13E0F15000401040E1F755
:100C200035C18C2F0E943F0536C18C2F8695869545
:100C3000837019F0813061F02EC1112321F08D2FC6
:100C40009C2F937002C080E090E00E942A182BC174
:100C5000112321F08D2F9C2F937002C080E090E033
:100C60000E94401820C18D2F112319F00E94AC134F
:100C700002C00E9407140E947E1415C18C2F83703D
:100C800009F047C011110BC12D2F22952695277011
:100C9000220F220F6D2F6F70862F90E0A0E0B0E042
:100CA000022E04C0880F991FAA1FBB1F0A94D2F7F7
:100CB000D4FF10C04FE050E060E070E004C0440F8B
:100CC000551F661F771F2A95D2F74095509560955E
:100CD000709503C040E050E0BA01C695C695C37058
:100CE0008A019B01082B192B2A2B3B2BC901B80128
:100CF000C23049F058F4C13019F00E944708CFC003
:100D00000E943508CCC00E945908C9C00E9433080F
:100D1000C6C0112319F08C2F817001C086958823DD
:100D200009F4BDC02D2F229526952770220F220F82
:100D30006D2F6F70862F90E0A0E0B0E0022E04C00F
:100D4000880F991FAA1FBB1F0A94D2F7D4FF10C0A7
:100D50004FE050E060E070E004C0440F551F661F94
:100D6000771F2A95D2F7409550956095709503C0EE
:100D700040E050E0BA01C695C695C3708A019B0158
:100D8000082B192B2A2B3B2BC901B801C23049F083
:100D900058F4C13019F00E940C0981C00E94FA0871
:100DA0007EC00E941E097BC00E946D0878C0CF7073
:100DB000112339F08C2F0E9493088D2F0E94380543
:100DC0006EC08D2F0E943F058C2F0E94B40867C013
:100DD000D23F21F128F4D03F41F0D13FC1F043C0D0
:100DE000D33F19F1D43F79F03EC0112341F00530D3
:100DF00008F051C08C2F8F710E94D9084CC006306A
:100E000008F049C0F7CF8091C70282FF18C01123B4
:100E100039F08C2F8F710E9493083DC01123C9F3C4
:100E20008C2F8F710E94B40836C0112329F08C2FAB
:100E30008F710E947E082FC00E9479082CC0112358
:100E400049F0CF718C2F0E94930863E08C2F0E9491
:100E5000B50D21C081E00E94D00D0230E0F082E0AB
:100E60000E94D00D18C0112331F0002391F28D2F74
:100E70000E94060410C0002399F2D93349F41FEFF1
:100E800027EE33E0115020403040E1F700C0000071
:100E90008D2F0E94B00488EF8C0D843020F40E94C6
:100EA00005180E949B03DD20C9F00E94230D80FDE0
:100EB00015C0F70112820E941D0D0E949308C70100
:100EC0000E948F070E941D0DDF91CF911F910F91FE
:100ED000FF90EF90DF90CF900C94B408DF91CF910A
:100EE0001F910F91FF90EF90DF90CF9008950F9397
:100EF0001F93CF93DF93EC01688179818A810E94EF
:100F0000D5098C010E9430090E942108B801CE0148
:100F10000E944605DF91CF911F910F910895CF93C5
:100F2000DF93EC01988189812B813C81232B31F067
:100F30008F3F31F481E09F3F19F403C081E001C08D
:100F400080E080FD1DC0CE010E943903811110C0D8
:100F50000E94270D8823A1F08A81882389F080913F
:100F6000C70282FD0DC082E0DF91CF910C94D00DBD
:100F7000CE010E947707CE01DF91CF910C941A0326
:100F8000DF91CF91089580E090E00E942A1880E0E0
:100F900090E00E9440180E944E0D0E94700D0E9429
:100FA000AF150C947E1480910201909103010E9470
:100FB0009C180C94C3070E943E0D0C94D307929585
:100FC0009F70963079F010F4925001C09A50923090
:100FD00068F4803F69F018F4883E40F409C0843F0B
:100FE00029F406C0883E20F0813F11F080E008958A
:100FF00081E00895FC01808191810E94CA090E94CC
:10100000DF070895CF93DF9300D000D01F92CDB7B4
:10101000DEB70F900F900F900F900F90DF91CF9150
:101020000895CF93DF9300D000D000D0CDB7DEB7C6
:1010300026960FB6F894DEBF0FBECDBFDF91CF91DD
:101040000895089508950C9422080C9423080E9492
:1010500025086093B2017093B3018093B40190931B
:10106000B5010C94C3070C9427080F931F930091AC
:10107000B2011091B3012091B4013091B501602B00
:10108000712B822B932B1F910F910C9427080F9398
:101090001F930091B2011091B3012091B4013091DE
:1010A000B50160237123822393231F910F910C9428
:1010B00027080F931F930091B2011091B301209163
:1010C000B4013091B50160277127822793271F91C2
:1010D0000F910C9427080C9422080E946B086093CF
:1010E000AE017093AF018093B0019093B1010C9465
:1010F000C30760E070E0CB010C946D080F931F9361
:1011000041E050E060E070E08A019B0104C0000F04
:10111000111F221F331F8A95D2F7C901B8011F91F1
:101120000F910C946D080F931F9341E050E060E025
:1011300070E004C0440F551F661F771F8A95D2F7D1
:101140008091AE019091AF01A091B001B091B10139
:101150008A019B01082B192B2A2B3B2BC901B801B3
:101160001F910F910C946D080F931F9341E050E075
:1011700060E070E004C0440F551F661F771F8A951A
:10118000D2F740955095609570958091AE01909101
:10119000AF01A091B001B091B1018A019B01082378
:1011A00019232A233B23C901B8011F910F910C94E5
:1011B0006D080F931F9341E050E060E070E004C0C1
:1011C000440F551F661F771F8A95D2F78091AE0195
:1011D0009091AF01A091B001B091B1018A019B0142
:1011E000082719272A273B27C901B8011F910F910A
:1011F0000C946D080F931F930091AE011091AF01F5
:101200002091B0013091B101602B712B822B932B77
:101210001F910F910C946D080F931F930091AE01D5
:101220001091AF012091B0013091B1016023712381
:10123000822393231F910F910C946D080F931F939A
:101240000091AE011091AF012091B0013091B10138
:1012500060277127822793271F910F910C946D08A7
:1012600008952BE0929F800D1124E82FE695E695D6
:10127000E695877051E001C0550F8A95EAF785E041
:10128000E89FF0011124E057FE4F20E030E070E0CD
:101290004081CB01022E02C0969587950A94E2F711
:1012A0008170819584278523842781932F5F3F4F09
:1012B0002530310569F708952BE0929F800D1124A8
:1012C000682F669566956695982F977085E0689F5C
:1012D000B001112440E050E080E0FB01E40FF51F75
:1012E000E057FE4F208130E0092E02C03695279549
:1012F0000A94E2F721703327042E01C0220F0A94CA
:10130000EAF7822B4F5F5F4F4530510531F7089563
:10131000BF92CF92DF92EF92FF920F931F93CF93E2
:10132000DF938C01C090AE01D090AF01E090B0018E
:10133000F090B1018091B2019091B301A091B401FC
:10134000B091B501C82AD92AEA2AFB2ACFE1D0E018
:10135000D701C6010C2E04C0B695A7959795879521
:101360000A94D2F780FD04C0219790F7B12C07C0F2
:10137000BC2EB8018C2F0E94C2100197A9F38B2DAF
:10138000DF91CF911F910F91FF90EF90DF90CF9061
:10139000BF900895CF93DF93EC010E948809BE01AE
:1013A0000E94C210DF91CF9108951F93CF93DF93D6
:1013B000EB0190918F01992321F0CB010E94CA0982
:1013C00013C0882349F0CB010E948809182F682F89
:1013D000CE010E94310904C0CB010E945C09182F84
:1013E000BE01812F0E94C210DF91CF911F910895FD
:1013F0001F93CF93DF93C091B60116E08091B701A0
:10140000C81799F0D0E01C9FF0011D9FF00D11242A
:10141000E854FE4F408151816281738184819581BE
:101420000E9411082196C770E9CFDF91CF911F91DB
:1014300008954091E8015091E9016091EA017091AD
:10144000EB018091EC019091ED010C941108EF9269
:10145000FF920F931F93CF93DF938091ED018295BD
:101460008F7009F065C08091EA01882309F460C09B
:101470008091B601F090B7011091E8010091E90167
:101480006091EB017091EC0191E01F3F09F090E059
:10149000C0910001D0910101292F96E0E92E8F150E
:1014A00009F446C06115710521F00F3F21F030E0CD
:1014B00003C031E001C0322F90E030FD36C0E89E1D
:1014C000F001E99EF00D1124DF01A854BE4F1196E2
:1014D0003C911197301329C03C91311326C01296CC
:1014E0003C911297311121C013964D915C91149744
:1014F000461B570B4C175D07C0F48091ED018F70B0
:1015000080618093ED01E354FE4F80818F70806194
:10151000808388EE91E00E948F07DF91CF911F9129
:101520000F91FF90EF900C94F80901968770B7CF58
:10153000DF91CF911F910F91FF90EF9008959F92AF
:10154000AF92BF92CF92DF92EF92FF920F931F93D1
:10155000CF93DF93CDB7DEB761970FB6F894DEBFB8
:101560000FBECDBF8C0185E0F801DE011D96019014
:101570000D928A95E1F7D8011296EC909091E801CE
:10158000E091E9012091EB013091EC012115310549
:1015900031F0EF3F31F481E09F3F19F403C081E067
:1015A00001C080E0B82FB1709B2E80FD47C1D801EB
:1015B0004C9111965C9111971396AD90BC90149735
:1015C00088EEC82E81E0D82EF090EA01B501621BAA
:1015D000730B2091000130910101FF2009F4D9C063
:1015E0008091ED016217730708F095C0282F207FC6
:1015F00009F052C05E1313C0491311C0FE2CE11054
:101600000EC08F7080618093ED010E94190AC6019F
:101610000E948F078091ED01F80185834DC1AB28B1
:1016200031F05F3F31F481E04F3F19F403C081E0B6
:1016300001C080E080FD03C081E08E2502C080E013
:1016400090E0F82FF170FF2E80FF1CC08091B60152
:101650002091B70136E0821709F40BC190E0389F62
:10166000F001399FF00D1124E854FE4F61815613AB
:1016700006C06081461303C06281E61203C0019672
:101680008770E9CFFE2CEE2009F416C18091ED01A0
:1016900081608093ED0154C05E1306C0491304C0FD
:1016A000E11002C0F80199C0C8010E94FA0788231E
:1016B00061F1EE2051F12091ED01822F82958F7022
:1016C00090E0029774F08091E8019091E901988789
:1016D0008F831986BB86AA862C87CE0107960E9427
:1016E0008F0786E0F801A8EEB1E001900D928A958F
:1016F000E1F70E94270A0E94190A0AC05E1711F139
:10170000C8010E94FA0781112CC0C8010E948F07EE
:10171000FF24F394D1C0282F207F81F77A2DB98A36
:10172000A88A6E2D89890E94020888EE91E00E94A5
:101730008F0786E0D6011D928A95E9F70E94190A63
:10174000F12CBAC04913DCCFE110DACFF801858360
:10175000C8010E948F0786E0D6011D928A95E9F79D
:10176000ABC0EE2091F22091ED01822F82958F7017
:1017700090E002970CF4B5CF8091E8019091E901D7
:101780009A8389831B82BD82AC822E83CE0101960F
:10179000A6CF6217730708F044C0FE2CEE2009F4B0
:1017A000B4CF5E1330C049132EC02091ED0120FD4F
:1017B00021C0822F82958F70482F50E0411551052E
:1017C000C9F0F80125834F30510541F08F5F982F04
:1017D0009295907F822F8F70892B8583C8010E94FC
:1017E0008F0786E0F801A8EEB1E001900D928A958E
:1017F000E1F73CC086E0F801A8EEB1E001900D925F
:101800008A95E1F759C0C8010E94FA07811169CF92
:101810008091ED0181608093ED01C8010E948F07E6
:101820004BC07A2DB98AA88A6E2D89890E94020838
:1018300086E0D6011D928A95E9F718C0EE2009F4DA
:1018400064CFC8010E94FA07F82E882309F45DCFFF
:1018500086E0F801A8EEB1E001900D928A95E1F7DB
:1018600088EE91E00E9400040E94270A0E94190A53
:1018700023C04D875E878D859E850E94CA09292FCA
:1018800022952F70223028F49F7039F0811105C005
:101890000BC0243028F49F7049F4805E883020F01B
:1018A000C8010E948F079F2CF92C06C0D8011596FD
:1018B0009C91907F91F7F8CF8F2D61960FB6F89499
:1018C000DEBF0FBECDBFDF91CF911F910F91FF9073
:1018D000EF90DF90CF90BF90AF909F9008951F93AF
:1018E000CF93DF93CDB7DEB72C970FB6F894DEBF5A
:1018F0000FBECDBF4F83588769877A878B879C87B8
:10190000CE0107960E949F0A8823D1F09F81888587
:101910002A853B85232B31F08F3F31F481E09F3FB7
:1019200019F403C081E001C080E080FD47C04F8111
:10193000588569857A858B859C850E9411083EC0F3
:1019400086E0FE013796DE01119601900D928A9590
:10195000E1F7FF81E8856A857B856115710531F0C6
:10196000EF3F31F481E0FF3F19F403C081E001C093
:1019700080E080FD23C02091B70130E0C9010196CD
:10198000877099274091B60150E084179507F1F1CF
:10199000F983EA837D836C8396E0929FD001939FC5
:1019A000B00D1124A854BE4FFE01319601900D9246
:1019B0009A95E1F78093B7010E94F80916E08091AB
:1019C000B6019091B701891771F1189FC0011124D8
:1019D00088549E4F0E949F0A882329F1E091B60106
:1019E0001E9FF0011124E854FE4F40815181628115
:1019F0007381848195810E9411088091B60190E0E5
:101A00000196877099278093B601D9CF0E94DB0792
:101A10001092B7011092B601E8EEF1E086E0DF0126
:101A20001D928A95E9F72C960FB6F894DEBF0FBE8B
:101A3000CDBFDF91CF911F9108958091F6018595DB
:101A40008595859508958091F60187700895909108
:101A5000F601977081E009F480E008958091010219
:101A6000089590910102892B809301020895809539
:101A7000909101028923809301020895109201023E
:101A8000089590910002892B80930002089580951B
:101A90009091000289238093000208951092000221
:101AA00008958091F701089508950C94540D0C94B5
:101AB000550D9091C70292FD08C09091F7019817BB
:101AC00021F08093F7010C94570D08958091F70150
:101AD000882329F01092F70180E00C94570D0895A7
:101AE000CF93DF93E0910201F09103018091010215
:101AF0008083E0910201F0910301908180910002C6
:101B0000892B80838091F701882381F0E091020185
:101B1000F09103019081892B808380910201909143
:101B200003010E94561881110E94660DC0910201A6
:101B3000D091030148E050E06EEE71E0CE010E94CA
:101B4000BD1C892B69F088E0FE01AEEEB1E001908A
:101B50000D928A95E1F7CE01DF91CF910C94111887
:101B6000DF91CF9108950C94540D9091C70292FD8E
:101B700010C098E0899F90011124262B2093F60134
:101B80000E9493088091F6018595859585950C9422
:101B9000B30D0C9493081092F60180E00C94B30DF1
:101BA0002091F601809582238093F601982F9770FB
:101BB00099F430E0482F082E000C550B24173507F8
:101BC00059F09091C70292FD07C08595859585953E
:101BD0000E94B4080C94CB0D08959091C70292FB1B
:101BE000222720F9281769F080FB92F99093C70209
:101BF0008091C6029091C7020E94350E82E00C943B
:101C0000D00D08958091C70282FB882780F991E06A
:101C100089270C94ED0D81E00C94ED0D80E00C947F
:101C2000ED0D80E090E00E94D21C21E0893E9E4FA5
:101C300009F020E0822F089582E090E00C94CA1C05
:101C400083E090E00C94CA1CCF9384E090E00E9463
:101C5000CA1CC82F82E290E00E94CA1C2C2F30E0E0
:101C6000A901582BCA01CF910895CF93C92F682F8E
:101C700084E090E00E94D81C6C2F82E290E0CF912B
:101C80000C94D81CAB01BC018FE090E00C94EA1CD2
:101C9000AB01BC0183E190E00C94EA1C60E070E0D1
:101CA000CB010C94480E60E070E0CB010E94420E24
:101CB0000C944E0E69EE7EEF80E090E00E94F61CE0
:101CC00060E082E090E00E94D81C60E083E090E059
:101CD0000E94D81C1092B2011092B3011092B4016C
:101CE0001092B50160E084E090E00E94D81C60E0B2
:101CF00082E290E00E94D81C60E085E090E00E94C3
:101D0000D81C60E086E090E00E94D81C6FEF87E06E
:101D100090E00E94D81C40E050E0BA0188E090E0DA
:101D20000E94EA1C60E08DE090E00E94D81C40E038
:101D300050E0BA0188E190E00E94EA1C60E087E18F
:101D400090E00E94D81C40E050E0BA018CE190E0A5
:101D50000E94EA1C60E070E080E290E00E94F61CC5
:101D600040E050E0BA0188E190E00E94EA1C0C9447
:101D7000530E0C945A0E682F8EE090E00C94D81CF1
:101D80000E94311960930E0270930F02809310022B
:101D90009093110260930A0270930B0280930C02DD
:101DA00090930D02089581E008950C94D30E089548
:101DB0000C94D70E0C94D70E0C94DA0E0C94D70E0C
:101DC0000C94DE0E0C94D70E8EE991E10E94FB1765
:101DD0000E94E20E0C94E00E0E94D80E0C94D70ED6
:101DE0000E94A1110C949A030E941C190E94861251
:101DF0000E94F00E0C94DC0E5F926F927F928F9295
:101E00009F92AF92BF92CF92DF92EF92FF920F9389
:101E10001F93CF93DF93CDB7DEB72A970FB6F89411
:101E2000DEBF0FBECDBF0E949B12C82E81110E9443
:101E3000C00E32E0832E32E0932E00E010E0502EF0
:101E4000802F0E94C5115C01F401619071904F01D7
:101E50006826792661147104B1F40F5F1F4F0430B6
:101E6000110569F78FEF89838A831B820E942519E8
:101E70008160782F9D838C8349815A816B818D810C
:101E80000E94B6033AC08091120281FD0E94CE11D9
:101E9000D12CEE24E394F12CC3018E219F21892BB8
:101EA00029F10E94D50E8823A9F0DE825F82AE2040
:101EB000BF2081E0AB2809F480E088870E942519C3
:101EC0008160782F9A8789874E815F8168858A85AE
:101ED0000E94B603000F111FF801EE5FFD4F8081D5
:101EE0009181E826F926F182E08207C0D394EE0CB6
:101EF000FF1CFBE0DF12D0CFB0CF81E0C11001C0EA
:101F000080E02A960FB6F894DEBF0FBECDBFDF91FA
:101F1000CF911F910F91FF90EF90DF90CF90BF90E6
:101F2000AF909F908F907F906F905F9008950E94E8
:101F3000FC0E0E949C140C94AB03CF93DF930E9481
:101F4000C710EC01811521E5920708F045C0811505
:101F500030E5930708F094C0883E910528F5803E4F
:101F6000910508F0F8C0883A910570F4853A91051A
:101F700008F07CC08130910509F475C008F4E8C010
:101F8000049708F0E8C0E4C08F3B910508F0E0C07A
:101F9000C85AD0E0CC0FDD1FC55BDE4F0990D88159
:101FA000C02DCE019464D8C0811540E2940758F446
:101FB000811551E0950708F0CEC08D3E910508F4DB
:101FC000C7C09065C9C0C11580E4D80708F4C0C077
:101FD000DF70CE01906AC0C0811525E59207A8F494
:101FE000811534E5930708F095C0811543E5940702
:101FF00008F07BC0811552E5950708F061C0D82F25
:10200000CC27CE01816F906AA7C0C11589E5D8079A
:10201000A0F4C11528E5D20708F082C0C11536E545
:10202000D30708F095C08C2F0E945B118F7190E050
:10203000D82FCC27CE0190628FC0C1154AE5D407B6
:1020400008F474C0CE0190568115904208F080C00B
:102050008D2F8F710E945B11DD27D0628F71AE01D1
:10206000582BCA0179C081E090E076C0C55AD0E013
:10207000C758DE4F8881C82FD0E0CE0190646CC075
:1020800074E0969587957A95E1F7282F23703C2F79
:10209000337081E090E002C0880F991F3A95E2F713
:1020A0009C68AC01522B9A019C2F9F709695969537
:1020B00050E2959FE0011124C9018C2B9D2B4CC04F
:1020C0008370992721E030E002C0220F331F8A95E8
:1020D000E2F79C2F9695969580E2989FE001112457
:1020E000C22BD32BCE019C6837C08370992721E087
:1020F00030E002C0220F331F8A95E2F79C2F96959D
:10210000969540E2949FE0011124C22BD32BCE017F
:102110009A6822C0D82FCC27CE01846F906A1CC049
:10212000DC2FCC27CE01806F906A16C08C2F8F7069
:102130000E945B1194E0D695C7959A95E1F7CF7010
:10214000D0E0DC2FCC27D0699E01282BC90104C028
:1021500080E090E001C0CE01DF91CF9108952CE2A4
:10216000829FC0011124FC012BE0729FE00DF11D44
:102170001124E60FF11DEE0FFF1FE058FF4F859170
:10218000949108950E94AF100E949D0F0895823887
:10219000910569F1B0F48133910509F46DC048F4FB
:1021A0008932910509F463C08A32910509F469C046
:1021B00008958533910509F455C089339105B9F027
:1021C0000895833E910569F138F4803E9105B1F0A0
:1021D000823E910509F10895863E9105A9F1873E59
:1021E0009105B9F1843E910509F064C023C02091A6
:1021F000C60220FD4FC021FD4DC008958091C6024A
:1022000080FD44C08091C70280FF44C08091C60217
:1022100084FD42C083EE4DC08091C60282FF38C06B
:10222000F5CF8091C60282FD33C08091C70280FD48
:1022300031C0ECCF8091C70281FF32C08091C602CD
:1022400084FD2AC087EE35C08091C60283FF26C078
:10225000F5CF8091C60283FD21C08091C70281FD28
:102260001FC0ECCF8091C60285FD1CC01DC08091AF
:10227000C60285FD19C016C08091C60286FD16C033
:1022800017C08091C60286FD13C010C089E311C03B
:1022900082EE0FC080EE0DC080E00BC086EE09C05C
:1022A00084EE07C089E205C085E303C08AE201C06D
:1022B00081E390E008959091C60292FF0DC0282F0F
:1022C0002871283019F4877F846006C0282F247174
:1022D000243011F48B7F886093FF0DC0282F287164
:1022E000283119F4877E846106C0282F2471243197
:1022F00011F48B7E88612091C70220FF0DC0382F1A
:102300003871383019F4877F816006C0382F3171F9
:10231000313011F48E7F886021FF0DC0282F287185
:10232000283119F4877E816106C0282F217121315F
:1023300011F48E7E886194FD877E089580E0089573
:1023400008950E94110E811102C00E94B90E0E94D0
:102350001C0E809312020E94240E9093C702809359
:10236000C6020E94A0110E94200E682F70E080E03B
:1023700090E00E9433086091AE017091AF018091AE
:10238000B0019091B1010C946B08E82FF0E0EE0FD2
:10239000FF1FE053FD4F808191810895089580EAE9
:1023A0008A95F1F7089500C008950C94CF1108950F
:1023B0000C94D7110C94D8110C94D7110C94DC11F7
:1023C000F894E82FE295EF70F0E031A1282F2F70FC
:1023D00081E090E001C0880F2A95EAF7982F909548
:1023E000932391A392A1892B82A3789408950F93AC
:1023F0001F93CF93DF93C7E8D1E089918F3F11F00E
:102400000E94E01181E0CB38D807B9F7CCE7D1E0E2
:1024100007E811E089918F3F11F00E94E0110C173D
:102420001D07C1F7DF91CF911F910F910895BF92C2
:10243000CF92DF92EF92FF920F931F93CF93DF9390
:102440008C01C62FD0E0CE0189579E4F6C01FC0154
:1024500090819F3F09F450C0B62EF894E92FE29581
:10246000EF70F0E081A19F7021E030E001C0220F09
:102470009A95EAF7822B81A382A12095282322A393
:1024800078940E94D311ECE7F1E047E851E021E0B5
:1024900030E0E12CF12C61916F3F89F0A62FA295DD
:1024A000AF70B0E090968C9190E06F7002C09595FF
:1024B00087956A95E2F780FD02C0C90102C080E0FD
:1024C00090E0E82AF92A220F331F4E175F0719F709
:1024D000F60180818F3F11F00E94E01161E0E1146C
:1024E000F10409F460E08B2D0E94D511CC0FDD1FA3
:1024F000C00FD11FF982E882DF91CF911F910F9118
:10250000FF90EF90DF90CF90BF9008950E94F71159
:1025100088E0E0EDF2E0DF01982F1D929A95E9F74F
:10252000E8ECF2E0DF011D928A95E9F784E00E9471
:10253000E6120C942503FF920F931F93CF93DF9322
:10254000CDB7DEB728970FB6F894DEBF0FBECDBF6C
:102550008E010F5F1F4F88E0F80111928A95E9F70D
:10256000F12C6F2DC8010E941712F394F4E0FF12B2
:10257000F8CF48E050E0B80188EC92E00E94BD1C22
:10258000FF24F394009709F4F12C892B41F088E0A3
:10259000F801A8ECB2E001900D928A95E1F72F2D99
:1025A00044E060ED72E088EC92E00E94E7120E9445
:1025B00027038F2D28960FB6F894DEBF0FBECDBF30
:1025C000DF91CF911F910F91FF9008950895FF9291
:1025D0000F931F93CF93DF93F82E092F162FD72F2A
:1025E000C42F222349F081E0809315020E9425190F
:1025F0009093140280931302809115028823D9F0DE
:1026000080911302909114020E943D19059798F051
:10261000EF2DF02FA12FBD2F80E090E04C2F50E048
:102620008417950734F4219131912D933D930196B0
:10263000F7CF10921502DF91CF911F910F91FF906C
:1026400008950E9497190E94F40E0C94A8190E94F4
:10265000C3180E9487190E94E40E0E9421130E9451
:10266000B6190E94EC0EFBCF80911C0280FF06C0C1
:102670006091090170E0660F771F26C081FF04C0DA
:102680006091090184E005C082FF07C060910901E3
:1026900088E0689FB001112417C090911B02992314
:1026A000D1F060910801961788F72091090188E020
:1026B000289F90011124929FA001939F500D1124F7
:1026C00070E0CA010E948F1C6038710540F46115EA
:1026D000710519F406C068E070E0862F08958FE751
:1026E000089581E0089580911C0280FF08C06091E8
:1026F000050170E0759567957595679521C081FF17
:1027000006C06091050170E07595679519C082FF5C
:1027100004C06091050170E010C090911A029923E5
:1027200099F0609104019617A0F780910501899FA7
:10273000C001112470E00E948F1C6038710540F4C4
:102740006115710519F406C061E070E0862F0895E7
:102750008FE7089581E008958D3E21F40E9434139F
:10276000819504C08E3E29F40E9434138093200288
:1027700008958F3E21F40E943413819504C0803F58
:1027800029F40E94341380931F020895893F19F49D
:102790000E94731305C08A3F31F40E947313819520
:1027A0008093210208958B3F21F40E947313819539
:1027B00004C08C3F29F40E94731380932202089571
:1027C0009FE0980F983078F421E030E0A90102C032
:1027D000440F551F9A95E2F7CA0190911E02892B6A
:1027E00080931E0208958D3F21F480911C02816028
:1027F0000BC08E3F21F480911C02826005C08F3F88
:1028000029F480911C02846080931C0208958D3EFF
:1028100039F49091200297FF35C01092200259C0E0
:102820008E3E29F4909120021916BCF32BC0909192
:102830001F028F3E29F497FF25C010921F0249C046
:10284000803F19F41916CCF31DC090912102893FE5
:1028500029F41916BCF4109221023BC08A3F19F4E6
:1028600097FF10C0F8CF8B3F39F49091220297FF69
:1028700009C0109222022DC08C3F21F490912202B7
:102880001916BCF39FE0980F983080F421E030E0F7
:10289000A90102C0440F551F9A95E2F7CA0180951D
:1028A00090911E02892380931E0213C08D3F21F454
:1028B00080911C028E7F0BC08E3F21F480911C0200
:1028C0008D7F05C08F3F29F480911C028B7F809300
:1028D0001C0280911F02811106C08091200281118B
:1028E00002C010921B0280912102811106C08091CA
:1028F0002202811102C010921A0208950E94251925
:1029000020911F02211104C020912002222321F0D6
:10291000909319028093180220912102211104C082
:1029200020912202222321F0909317028093160215
:102930008DE192E00C941C18EF92FF920F931F937D
:10294000CF93DF9300D000D000D0CDB7DEB786E0C4
:10295000EDE1F2E0DE01119601900D928A95E1F72A
:10296000E0901F02F09020020091210210912202BB
:1029700010921F0210922002109221021092220245
:10298000E11003C0FF2009F45DC08091180290910E
:1029900019020E943D19AC0190911B02992339F054
:1029A00020910A0130E02417350758F04BC02091E0
:1029B0000B018AE0289F900111242417350718F095
:1029C00041C09F3F19F09F5F90931B02EE2061F082
:1029D0000E9434131E1414F09FEF01C091E0989FE1
:1029E000902D112490931F02FF2061F00E94341358
:1029F0001F1414F09FEF01C091E0989F902D1124B7
:102A00009093200230911F023323E1F020912002A5
:102A10002223C1F045EB3403C0011124992319F09E
:102A200090931F0203C081E080931F0235EB2303C4
:102A3000C0011124992319F09093200203C081E072
:102A400080932002011103C0112309F45DC080911D
:102A50001602909117020E943D19AC0190911A0242
:102A6000992339F02091060130E02417350758F0FA
:102A70004BC0209107018AE0289F90011124241760
:102A8000350718F041C09F3F19F09F5F90931A02DD
:102A9000002361F00E947313101614F09FEF01C021
:102AA00091E0989F902D112490932102112361F0C1
:102AB0000E947313111614F09FEF01C091E0989FCC
:102AC000902D112490932202309121023323E1F0C2
:102AD000209122022223C1F045EB3403C0011124CE
:102AE000992319F09093210203C081E08093210281
:102AF00035EB2303C0011124992319F0909322028E
:102B000003C081E08093220280911F0281110BC0DB
:102B100080912002811107C080912102811103C0A0
:102B20008091220281110E947E14EB82FC820D832F
:102B30001E8386E0FE013196ADE1B2E001900D9278
:102B40008A95E1F726960FB6F894DEBF0FBECDBF8B
:102B5000DF91CF911F910F91FF90EF900895EDE1DC
:102B6000F2E086E0DF011D928A95E9F710921B02E0
:102B700010921A0210921C020895CF93DF93EC0179
:102B8000FB018281882309F43CC1C430FDE5DF07E5
:102B900060F4CB3F9CE5D90788F49E0122503C4568
:102BA0002431310508F02EC109C0C236EDE5DE073B
:102BB00029F0C63AFDE5DF0709F024C10E94240E82
:102BC0009093C7028093C602C1318CE5D80709F4FF
:102BD000C6C008F042C0C930ECE5DE0709F49BC06E
:102BE00000F5C5308CE5D80709F485C078F4C3300A
:102BF000ECE5DE0709F478C008F07AC0C230DC45A5
:102C000009F0F5C08091C6028160EFC0C7309CE535
:102C1000D90709F478C008F07AC08091C6028061B3
:102C2000E4C0CD30FCE5DF0709F487C058F4CB30B1
:102C30009CE5D90709F479C008F07BC08091C602F1
:102C400088606FC0CF30FCE5DF0709F480C008F072
:102C500082C08091C602877FC8C0CE3F9CE5D9075D
:102C600009F471C000F5C531FCE5DF0709F485C042
:102C700068F4C3319CE5D90709F475C008F095C024
:102C80000E94DB078091C6028F77AFC0CC3FFCE586
:102C9000DF07A9F108F054C0CB3FDC4509F0A7C01D
:102CA0008091C70240C0C230EDE5DE0709F489C05B
:102CB00058F4C1158DE5D80709F45AC008F069C069
:102CC0008091C70282602FC0C236EDE5DE0709F4AD
:102CD0007CC0C63AFDE5DF0709F481C0C330DD459D
:102CE00009F085C080E06EC08091C60282607DC020
:102CF0008091C60216C08091C602886076C080911D
:102D0000C70282604FC08091C60280626EC080910F
:102D1000C60280646AC00E94DB078091C602806898
:102D200064C0846062C081603DC08091C6028E7FB5
:102D30005CC08091C6028D7F58C08091C60216C0CB
:102D40008091C70218C08091C7028D7F2BC08091EF
:102D5000C6028F7E4AC08091C6028F7D46C0809198
:102D6000C6028F7B42C08091C602877F8B7F3DC0A9
:102D70008091C7028D7F8E7F15C08091C60282FB35
:102D8000222720F991E0922790FB82F990FB83F9AA
:102D90002CC08091C702982F909591708E7F892BBF
:102DA00090FB81F98093C70222C00E94DB078091CB
:102DB000C60287FB222720F991E0922790FB87F932
:102DC00014C081E00E94BB0E12C08091C60284FB39
:102DD000222720F991E0922790FB84F906C0809188
:102DE000C602982F909590FB80F98093C60280913F
:102DF000C6029091C7020E94350E0E94DB0780E058
:102E000001C081E0DF91CF910895CF93DF938631A8
:102E10009C4541F5EB010E942E0D982F8A8120914F
:102E2000020130910301882379F09A7A81E009F454
:102E300080E080932302911102C069E201C065E342
:102E4000C9010E9498180AC080912302811102C012
:102E500069E201C065E3C9010E949A180E94700DE1
:102E600080E001C081E0DF91CF9108950F931F931F
:102E7000CF93DF93C42FD22FFC0182818823C9F026
:102E8000409326020E9425199093250280932402E4
:102E900080E28C0F883008F057C0C77081E001C015
:102EA000880FCA95EAF7DF91CF911F910F910C948B
:102EB000380580912602481330C0809124029091F9
:102EC00025020E943D19883C910538F510E21D0F3E
:102ED000CD17B9F080E28C0F883040F4C77081E0E4
:102EE00001C0880FCA95EAF70E943F05183028F5FF
:102EF00081E09D2F977001C0880F9A95EAF70E9494
:102F00003805802F0E942F051830F0F4D77081E02B
:102F100001C0880FDA95EAF70AC080E28C0F88308A
:102F200098F4C77081E001C0880FCA95EAF7DF9175
:102F3000CF911F910F910C943F05802FDF91CF917E
:102F40001F910F910C942F05DF91CF911F910F913D
:102F500008950F939C01CB01243F4CE5340731F1D8
:102F600088F4293DFCE53F07D9F02A3D4CE53407BC
:102F700079F1283D3C45A9F506E221EE41EE68EDE8
:102F80007CE52BC0263FFCE53F07E1F0A8F0273F9A
:102F90003C4539F507E225EE46EE67EF7CE51DC0BE
:102FA00007E225EE45EE69ED7CE517C006E221EE6D
:102FB00040EE64EF7CE511C007E225EE44EE65EFDC
:102FC0007CE50BC006E221EE42EE66EF7CE505C033
:102FD00008E221E045EE6AED7CE50E94361780E0CC
:102FE00008C0FC018281882319F01092260201C0DA
:102FF00081E00F91089590938D0180938C01089545
:1030000090932C0280932B020895E0912B02F09173
:103010002C02309721F00190F081E02D099480E09E
:103020000895E0912B02F0912C02309721F002805C
:10303000F381E02D09940895E0912B02F0912C0288
:10304000309739F022E0DC012C930480F581E02DEB
:10305000099408952091290230912A0228173907EE
:1030600071F090932A0280932902E0912B02F09153
:103070002C02309721F00680F781E02D0994089505
:1030800020912702309128022817390771F0909378
:10309000280280932702E0912B02F0912C023097B6
:1030A00021F00084F185E02D09940895FC01329609
:1030B00097E080E0915029F021912223D9F38F5F8E
:1030C000F9CF0895662349F0FC01329608962191C4
:1030D000621729F0E817F907D1F780E0089581E039
:1030E00008959C01FC0132969FEF80E041914617C4
:1030F00089F09F3F19F4411101C0982F8F5F8630EE
:10310000A9F79F3F39F0F901E90FF11D97FDFA95F5
:103110006283089508959C012A5F3F4FFC0142811C
:10312000461301C01282019682179307B9F70895DA
:103130000C9471180C948B18029626E0FC011192E5
:103140002A95E9F7089508950C94A3180C94A418EF
:103150000C94A3180C94A3180C94A318CF930E945A
:10316000AA180E949B120E94A818C0E08C2F0E94EF
:10317000C511892B29F4CF5FC430C1F780E001C0AD
:1031800081E0CF91089508951F920F920FB60F928C
:1031900011248F939F93AF93BF9380912D02811140
:1031A00013C08091D8029091D902A091DA02B09117
:1031B000DB024196A11DB11D8093D8029093D902E4
:1031C000A093DA02B093DB02BF91AF919F918F91F0
:1031D0000F900FBE0F901F9018958091300288239A
:1031E00031F10E948B0310922D0220E488E190E0DF
:1031F0000FB6F894A895809360000FBE20936000EE
:1032000083B7817F846083BF83B7816083BF7894F5
:10321000889583B78E7F83BF0FB6F894A895809169
:103220006000886180936000109260000FBE089576
:103230000E94DB070C948F0382E084BD93E095BD70
:103240009AEF97BD80936E0008952FB7F894809100
:10325000D8029091D902A091DA02B091DB022FBF7F
:1032600008952FB7F8946091D8027091D902809197
:10327000DA029091DB022FBF08959C014FB7F894BA
:103280008091D8029091D902A091DA02B091DB022C
:103290004FBF821B930B089578941F920F920FB625
:1032A0000F9211248F939F93AF93BF938091D80275
:1032B0009091D902A091DA02B091DB020196A11D92
:1032C000B11D8093D8029093D902A093DA02B093F3
:1032D000DB02BF91AF919F918F910F900FBE0F9026
:1032E0001F90189598E088E10FB6F894A895809300
:1032F00060000FBE90936000A895F894D8E0CEEFE0
:1033000028E3299320E0299314BEFFCF08950E945B
:10331000251990932F0280932E0290E080E80FB63B
:10332000F89480936100909361000FBE08950E940D
:10333000741C539A80E0815041F0A895EFE9FFE0BA
:103340003197F1F700C00000F6CF539878940895B4
:103350000E949C1A0E9400182FEF80E792E02150F3
:1033600080409040E1F700C0000008958091030381
:10337000882389F0109203030E94251990932F024D
:1033800080932E02809130028823D1F11092300276
:103390000E94181911C080913002811111C08091D2
:1033A0002E0290912F020E943D19069728F081E08D
:1033B000809330020E94ED1880913002882301F141
:1033C0000E94ED180E94AE18882339F1F8942AB1B2
:1033D0005B9A822F8C608AB99BB18CE098279BB94D
:1033E0003FE748E391E0315040409040E1F700C0B2
:1033F00000009BB189278BB92AB95B98789408950E
:103400000E947D1B80910903882329F08091E702A7
:1034100084FD0E94970F0C94431A08958091C50271
:103420000895089590913602981307C020913402B0
:103430003091350226173707A9F080933602709332
:1034400035026093340280933102709333026093AB
:1034500032028091200384FF05C063E081E392E0A3
:103460000C94791B0895BC0184E00C94121ABC01E1
:1034700083E00C94121A2091200324FF03C066E01D
:103480000C94791B0895CF93DF93CAE0D0E080912C
:10349000E70284FF18C0809142029091430298177E
:1034A000E1F028E0829FC001112468E08C5B9D4F11
:1034B0000E94751B8091420290E001968F709927BF
:1034C000809342020AC00E947D1B8FE99FE0019712
:1034D000F1F700C000002197D1F6DF91CF91089558
:1034E000CF93DF93EC01A0914302B0E0CD010196B0
:1034F0008F70992720914202281779F093E0AA0F44
:10350000BB1F9A95E1F7AC5BBD4F98E0FE010190BF
:103510000D929A95E1F7809343020E947D1B0E94D1
:10352000431A88E0FE01AAE3B2E001900D928A9569
:10353000E1F7DF91CF9108958CE091E00895FC01CF
:10354000808180768032A1F58181813061F484812F
:103550009581892B69F58AE392E090930503809326
:10356000040388E00895823041F484EC92E0909363
:1035700005038093040381E008958A3021F4838158
:103580008093C40215C0893099F48281938181159A
:10359000924081F484819581892B61F481E080934C
:1035A000390286819781909338028093370202C056
:1035B00080E008958FEF089520913702309138020E
:1035C000232B71F020913902213051F4FC018081CC
:1035D0008093C502109238021092370281E008955C
:1035E0008FEF08950895FC0193819330D9F068F42A
:1035F000913081F0923009F054C088E891E09093C6
:103600000503809304038BE30895913221F19232F4
:1036100091F147C083EC91E09093050380930403FC
:1036200082E108958281813071F028F08230C9F5FD
:1036300085ED91E00AC085EF91E0909305038093BA
:10364000040384E0089585EE91E090930503809350
:1036500004038EE008958281882329F0813009F5E2
:1036600083EB91E002C08AE991E090930503809397
:10367000040389E0089584819581009751F00197B2
:1036800081F489EF91E090930503809304038BE725
:10369000089584E792E0909305038093040380E407
:1036A000089580E008951F93CF93DF93162FEA01CA
:1036B000288124FF05C0398128E82327298302C0F7
:1036C0002AE52883212FFC01CE010296DC013191ED
:1036D0003D9321501216DCF3612F0E948E011C5F76
:1036E0001883DF91CF911F91089547EE52E00C941B
:1036F000531B40E253E00C94531BCF93DF93609134
:103700000603635067FD93C080910203CCE0D0E0D4
:10371000C81BD109C65FDC4F80910103803120F4C2
:10372000CE010E94F21A81C08D3209F06EC068305D
:1037300009F07BC083EC8093DC028AE58093190159
:10374000109200038881807621F0CE010E949F1A9A
:1037500049C09A811092E5028981811106C01092B8
:10376000E60225EE32E082E038C0853019F490930D
:10377000070330C08630A1F48B81813041F0823064
:1037800031F0833021F0813211F0823221F4CE0108
:103790000E94F31A01C080E090E49093000322C0DD
:1037A000883089F0893019F49093090313C08A3066
:1037B00069F08B3079F48BE48093E80280932103E5
:1037C0008093F40207C029E033E002C025EE32E026
:1037D00081E003C025EE32E080E0309305032093C2
:1037E000040309C08F3F39F4988197FD8E8190E8DA
:1037F0009093000307C09F81911104C09E81981788
:1038000008F4892F8093180110C08091000387FF6E
:103810000CC0CE010E94DC1A8F3F21F48EE1809310
:10382000190103C0811110921801109206038091B2
:10383000190184FF4CC0809118018F3F09F447C0E3
:10384000C82F893008F0C8E08C1B80931801909134
:10385000DC0288E889278093DC02CC2359F180912F
:103860000403909105032091000326FF12C0ACEDE4
:10387000B2E02C2FAC014C5D5240FA01EA0FFB1F65
:10388000E4911196EC931197215011962111F5CFE7
:1038900008C0EDEDF2E0DC012C2F3D913193215079
:1038A000E1F701962FEF2C0F820F911D90930503E6
:1038B000809304036C2F8DED92E00E948E01CC5F0B
:1038C000CC3019F08FEF80931801C093190184E177
:1038D00099B19C7031F48150D9F71092070310927E
:1038E000FF02DF91CF910895CF93DF93E9E6F0E0F7
:1038F000808188608083E99AC7EED2E08BE4898377
:10390000A0E2B3E011968C931197E3EFF2E081838C
:103910008AE588838C938083DF91CF91089597FB0C
:10392000072E16F4009407D077FD09D00E94A91C39
:1039300007FC05D03EF4909581959F4F08957095B2
:1039400061957F4F0895EE0FFF1F0590F491E02DD4
:103950000994AA1BBB1B51E107C0AA1FBB1FA617D6
:10396000B70710F0A61BB70B881F991F5A95A9F728
:1039700080959095BC01CD010895FB01DC0104C048
:103980008D910190801921F441505040C8F7881B57
:10399000990B0895F999FECF92BD81BDF89A9927A8
:1039A00080B50895A8E1B0E042E050E00C94FE1C20
:1039B000262FF999FECF92BD81BDF89A019700B4E8
:1039C000021639F01FBA20BD0FB6F894FA9AF99A88
:1039D0000FBE08950396272F0E94D91C0E94D81C61
:1039E000252F0E94D91C242F0C94D91C0196272F17
:1039F0000E94D91C0C94D81CDC01CB01FC01F99964
:103A0000FECF06C0F2BDE1BDF89A319600B40D922A
:0C3A100041505040B8F70895F894FFCFE3
:103A1C00C800F801280850011E0A14010E1A701A69
:103A2C003B1A371A331A111AFF5AE200E900EA005E
:103A3C00B500B600B700CD008301CC008A0192011D
:103A4C0094012102230224022502260227022A02C3
:103A5C00B300B4006F007000818283E200E900EAD9
:103A6C0000B500B600B700CD008301CC008A0192EE
:103A7C000194012102230224022502260227022A94
:103A8C0002B300B4006F007000818283309796956A
:0C3A9C0032316061626391343533940074
:00000001FF
